:020000040000FA
:02000000B52A1F
:080008009100030E92008B1A17
:100010002D280B1A1D28120E8300910E110E0900B7
:1000200081018316640088308100831285140130B9
:10003000860090308B00900108008B100C308C00F3
:100040008C0B202806180B28AD30810020308B0047
:100050000230900008308C000B280B11101940283A
:100060008C0803193928060C8D0C8C03AD308100E7
:100070000B28061C5A28013090000D088E005A28C3
:1000800090195A288C08031952288F0C031C4B28EE
:10009000000085144E288510000000008C03B53048
:1000A00081000B2800000000000085149015A83086
:1000B00081000B2810308B00013090050B28851033
:1000C000063090000000B5308100A0308B00083071
:1000D0008C00080018300605A100063006059F00B8
:1000E0002002031D7C2021082202031DA2201F08DC
:1000F000A0002108A200080020081F06063C0319E2
:10010000C8281F0DA006201994289708031D9228BF
:100110009808031D91281308970014089800970861
:100120000319980397030800970A0319980A1308FC
:100130001702031D080014081802031D0800970188
:100140009801080022082106183C0319C828210D2F
:10015000A206221ABA289908031DB8289A08031D76
:10016000B7281508990016089A00990803199A03E8
:1001700099030800990A03199A0A15081902031D20
:10018000080016081A02031D080099019A010800C8
:10019000A30A0800A022101CCA28101008005F2023
:1001A000A0229018D02808001508990016089A0077
:1001B00003109A0C990C1308970014089800031068
:1001C000980C970C0800CA200E089300CA200E084D
:1001D0009400CA200E089500CA200E089600D4206C
:1001E00072308F00CF200521C92A6521270895008C
:1001F0002608960065212708930026089400D4203D
:100200002A088F00CF200521C92A8B1200308900CF
:100210001308880083168801081555308900AA3014
:100220008900881488181229081283120130890065
:100230001408880083168801081555308900AA30F3
:100240008900881488182229081283120230890034
:100250001508880083168801081555308900AA30D2
:100260008900881488183229081283120330890003
:100270001608880083168801081555308900AA30B1
:100280008900881488184229081283128B160800E6
:100290000030890083160814831208089300013087
:1002A000890083160814831208089400023089001C
:1002B00083160814831208089500033089008316FA
:1002C000081483120808960008002C308400A90145
:1002D000A701A601A908031D8729CA200E08203CF2
:1002E00003196A290E08093C03196A290E080D3CF6
:1002F00003196A290E082B3C03196A290E082D3CA4
:1003000003196A290E088000A90A840A6D2984034A
:100310000030A4000130A500B221A90B90290800EB
:1003200084030030A4000A30A500B221A90B99294A
:10033000080084030030A4006430A500B221A90B9A
:10034000A229080084030330A400E830A500B221EC
:10035000A90BAB29080084032730A4001030A500A6
:10036000B22108002F300002A800A80BB82908000D
:100370002508A7070318A60A2408A607B5292308F5
:100380008F00CF20A301C92A2308303E8F00CF2041
:1003900030308F00CF2031308F00CF200D308F00D4
:1003A000CF20A301C92A2308A500A4017922A30113
:1003B000C92A17089B0018089C0019089D001A08F4
:1003C0009E001B088F00CF201C088F00CF201D0827
:1003D0008F00CF201E088F00CF20C92A17089B004E
:1003E00018089C0019089D001A089E002A08523C13
:1003F000031D022A961F022A1D08A5001E08A4003C
:100400004022122A1508A5001608A4000310A40C07
:10041000A50C25081D02031C9E03A50024081E022E
:10042000A400352209308F00CF202A08523C031D3A
:10043000212A941F212A1B08A5001C08A400402281
:10044000312A1308A5001408A4000310A40CA50C5D
:1004500025081B02031C9C03A50024081C02A40001
:1004600035220D308F00CF20C92AA41F402AA409AD
:10047000A509A50A0319A40A2D308F00CF20432A0D
:100480002B308F00CF206922080013088F00CF2067
:1004900014088F00CF2015088F00CF2016088F007A
:1004A000CF20C92A2B308F00CF201608A4001508B2
:1004B000A500692209308F00CF202B308F00CF207C
:1004C0001408A4001308A50069220D308F00CF2066
:1004D000C92A2730A6001030A7008E2228088F00D6
:1004E000CF200330A600E830A7008E2228088F0016
:1004F000CF200030A6006430A7008E2228088F008D
:10050000CF200030A6000A30A7008E2228088F00D6
:10051000CF202508303E8F00CF2008002F30A800C4
:10052000A80A2708A5022608031C013EA4020318F6
:10053000902A2708A50726080318013EA4070800EB
:100540006A20080056308F00CF2032308F00CF2035
:100550002E308F00CF2030308F00CF2030308F00F2
:10056000CF200D308F00CF2008008316FF3086008B
:100570000030850083128501102006300605A0009A
:1005800018300605A2004821A301D4204E30AB004C
:10059000A2228E01CA200E08793C0319D9290E081F
:1005A0007A3C0319E3280E08703C0319BF290E0892
:1005B000683C0319452A0E085A3C031DE22A2A30DA
:1005C000AA00F5280E08523C031DE92A5230AA0061
:1005D000F5280E08723C031DF02A5230AA00F528B7
:1005E0000E08483C0319522A0E08513C0319EE2903
:1005F0000E08503C0319C4290E08413C031D032B6F
:100600005930AB00C92A0E08613C031D0B2B2B0887
:100610008F00CF20C92A0E08713C0319D329C92A9B
:02400E00F93F78
:00000001FF
